S31508001800F8090020D9180008E7180008E9180008A0
S3150800181000000000000000000000000000000000BA
S315080018200000000000000000000000000119000888
S315080018300000000000000000031900083137000806
S31508001840DD410008071900080719000807190008EC
S3150800185007190008071900080719000807190008DA
S31508001860071900089528000807190008071900082D
S3150800187007190008071900080719000807190008BA
S3150800188007190008000000000000000007190008FA
S3150800189000000000071900080719000807190008C2
S315080018A0000000000719000807190008293C00086D
S315080018B007190008071900080719000800000000A2
S315080018C0EE11AA550348854600F0B2FC00480047C9
S315080018D0854F0008F80900200B4880F308880B4854
S315080018E080470B480047FEE704207146084202D0AD
S315080018F0EFF3098001E0EFF30880714603F042FA3E
S31508001900FEE7FEE7FEE7FEE7F8090020793800085B
S31508001910C518000830B50B460146002020220124D0
S3150800192009E00D46D5409D4205D31D469540491B05
S315080019302546954040191546521E002DF1DC30BD4E
S3150800194070B500242546002801DA01244042002902
S3150800195001DA01254942FFF7DDFFAC4200D04042DB
S31508001960002C00D0494270BD03460B439B0703D0A9
S3150800197009E008C9121F08C0042AFAD203E00B7846
S315080019800370401C491C521EF9D27047D2B201E0BE
S315080019900270401C491EFBD270470022F6E710B5BC
S315080019A013460A4604461946FFF7F0FF204610BDBF
S315080019B0F8B502464A40D40F42004B0052085B086D
S315080019C09A4202D20246084611464A0023D0C30D5F
S315080019D04A00DDB2120EAD1A202D35DA490201266B
S315080019E0490AF6058A19002C00D0524220214F1BBD
S315080019F01146B9402A411018C20D9A4221D0002C2E
S31508001A0017D0012D08DCDA05801AD20F8019D20703
S31508001A10DBB200F023FBF8BDDA05801A012340008B
S31508001A201B06C01880185A428018CA0F104349006E
S31508001A3007E04908C2071143DA05801A80194008E9
S31508001A40801800F003FBF8BD61000122511A001B43
S31508001A50F7E70122D2075140AAE70122D2075040F0
S31508001A60A6E7024670B54A40D30FDB0740002DD0E3
S31508001A704A002AD0010E140E000212020919400A61
S31508001A80520A8418E50104465443000A120A2E0431
S31508001A905043A4194219200CC543AA18120C012553
S31508001AA0AD03521C521912047F39240400D0521C6B
S31508001AB0104301D44000491EC2B20C06C0092018C2
S31508001AC0401C4008802A02D003E0002070BD400870
S31508001AD04000002900DA0020184370BD70B50246A0
S31508001AE04A40D50F40004A00ED0740085208002832
S31508001AF014D0002A12D0C40DD30D41020120C0050E
S31508001B005202490A520AE41A091812187D349142F7
S31508001B1001D3641C00E04900002C01DA002070BDE6
S31508001B200023914201D3891A03434008490000283B
S31508001B30F7D100290AD0914202D10121C90705E04F
S31508001B40914201D2012101E00121C943E005C018F3
S31508001B50401900F07BFA70BDF0B5074608465840B4
S31508001B6087B0C00F049048000E465900400849083F
S31508001B70BC1A884105D2384631461E4617460B46DA
S31508001B8002465800400810434CD0300D03904005DB
S31508001B905900400D490D0590401A0290402872DA06
S31508001BA018030121000B09050843019004980092C7
S31508001BB0002805D0019952420020884100920190E0
S31508001BC0029840210A1A0199009800F00BFA054676
S31508001BD00C466B4607CB00F026FAC0197141039AEA
S31508001BE00E0D0023D71756401A467A40164344D09E
S31508001BF0049A002A2DD0029A012A039A15DC1205A6
S31508001C00C01A914101263605001C7141D20F059E66
S31508001C10D2070093019202962A46234600F064FAF8
S31508001C2007B0F0BD38463146FAE71605224A0F4690
S31508001C30B218C01AB74101210905001C4F41001806
S31508001C407F41114618187941E20F10436D19644116
S31508001C5013E0E2076D0815436408C2071443039AA4
S31508001C6001261205C01A91413605001C7141CE079E
S31508001C70400830434908C01851412A46234600F017
S31508001C8026FACDE7FFE7049801224000C117121A89
S31508001C9000238B4104983146C417381AA141EEE750
S31508001CA030B40124E407634030BC55E730B401245E
S31508001CB0E407614030BC4FE70000E0FFF0B51FB411
S31508001CC088B00B990998002448400999C00F490023
S31508001CD049080991C0070B990090490049080B91DA
S31508001CE009990898A64608431CD00B990A980843F0
S31508001CF018D0099801244000420D4800410D099862
S31508001D0024050003000B204309900B980003000BE1
S31508001D1020430B9050181C49401800220190144685
S31508001D20104605E0002001460DB0F0BD032801DA93
S31508001D30034600E003239C46C11A0AAE0AE05F0088
S31508001D4008ADED5B4F00F75B7D430027AA187C4181
S31508001D50491C5B1E6145F2DD410004AB5A52210461
S31508001D60120C0A43240C401C0828DFDB0198029059
S31508001D700099704601910090059B049A0799069868
S31508001D8000F0B2F9D0E700000DFCFFFFF0B50C46F5
S31508001D905C4085B0E40FE40703944C000026640811
S31508001DA059009446490802460296224321D06246C3
S31508001DB00A431ED06200570D4A000E032303550D31
S31508001DC0012402462C492405781B1B0B360B4018A8
S31508001DD023432643614600901C46501AB44103D358
S31508001DE00098401C009002E0921800985B41002879
S31508001DF003DA0020014605B0F0BD002001210905DF
S31508001E000746864611E064461D46141BB54106D3AF
S31508001E106546521BB341744607430C43A646CD0795
S31508001E2040084908284392185B4105460D43EAD104
S31508001E301046184313D0604619465040714008436F
S31508001E4006D06046101AB34106D20122002306E0E6
S31508001E5000220123DB0702E00122D2435310009837
S31508001E6074460105381C6141029C039D00196941AD
S31508001E7000F02DF9BFE70000FD030000C217C10FEF
S31508001E80504010B54018CA079623002100F0E6F81E
S31508001E9010BD10B500229623114600F0DFF810BDDC
S31508001EA00EB5C217C10F5040CA0740180021054B8E
S31508001EB00293019200910A460B4600F015F903B009
S31508001EC000BD0000330400000EB50549029100214B
S31508001ED000910A460B46019100F006F903B000BDD1
S31508001EE033040000410040020122400AD205090ECF
S31508001EF080187F2901DA00207047962903DC96228C
S31508001F00511AC84070479639884070474A000903F5
S31508001F100123090B1B051943094B10B5520D9A42AB
S31508001F2001DA002010BD064B34339A4203DC9A1AB4
S31508001F3000F068F810BD03495118884010BD00002C
S31508001F40FF030000CDFBFFFFC20FD2074000400889
S31508001F500BD0C10D0723DB01C91840020905400A49
S31508001F601143C208400711437047002001467047D5
S31508001F7010B5002904DB0124E40740428C412146C0
S31508001F80002B04DB1C460123DB075242A3418B428C
S31508001F9000D1824210BD0000CB0FDB07490010B507
S31508001FA0490802460A4307D00A0D07240903E40133
S31508001FB0090B121B002A01DC002010BDC900440FC2
S31508001FC00C43C100E018D205801800F03FF810BD98
S31508001FD00122D207002800DB101A002900DB511A5B
S31508001FE08142704710B5202A04DB0146203A914009
S31508001FF0002010BD914020239C1A0346E340194354
S31508002000904010BD10B5202A04DB0846203AD0407F
S31508002010002110BD0B46D340D0402024A21A91407F
S315080020200843194610BD10B5202A06DBCB1708460B
S31508002030203A1041C1170B4306E00B461341D04026
S315080020402024A21A91400843194610BD002904DA33
S31508002050401C490001D140084000704770B4002474
S31508002060050C05D11024000402D1002921D0112421
S31508002070050E01D100020834050F01D10001241D07
S31508002080850F01D18000A41C002801DB4000641CD8
S31508002090002908D020252E1B0D46F540A14000D06A
S315080020A001212943084301061B1B000ADB1D02D533
S315080020B0002070BC7047DB05181880180029F8DA6C
S315080020C0401C4900F5D170BC40084000704710B567
S315080020D0002B08DA0024401C614192185B411A4320
S315080020E001D14008400010BDF0B51FB482B00546C6
S315080020F00C0003D0084602F0CDF802E002F0CAF858
S3150800210020300246009021462846FFF76BFF049BC5
S31508002110059A04460F4618431143084314D0184637
S3150800212010431BD0009840210A1A18460599FFF754
S3150800213069FF05460E46009A05990498FFF752FF6F
S31508002140084305D0012004E02046394607B0F0BD13
S315080021500020C11705430E432C43374300990E98B8
S315080021606305401A7905E40A00220C43FD0A0A3081
S3150800217002D500200146E9E70105101969410C9CC2
S315080021800D9D00196941FFF7A2FFDFE7FEB50023A1
S315080021901A461B1A8A4103DB0020014603B0F0BD2C
S315080021A04A000D0301212D0B0905520D0D43D107D8
S315080021B002D100186D41521E5110FF31FF31013115
S315080021C0002704463E4638460097019102460121FB
S315080021D000200905FFF716FFC3197141F8183246A2
S315080021E084468E464A4161462846611A904104D380
S315080021F06046241A954176461F46241900986D4173
S31508002200401C00903428E1DDF91930467041091B5D
S31508002210A84103D20022D243134601E00022134606
S3150800222001980105381C7141FFF751FFB6E7000018
S31508002230064C0125064E05E0E36807CC2B430C3C0B
S3150800224098471034B442F7D3FFF740FBFC64000804
S315080022501C65000810B50446002C08D10121092088
S31508002260C00600F0E3FD002000F0E6F852E0012C7D
S3150800227005D102210920C00600F0D8FD4AE0022C4B
S3150800228005D104210920C00600F0D0FD42E0032C48
S3150800229005D108210920C00600F0C8FD3AE0042C43
S315080022A005D110210920C00600F0C0FD32E0052C3A
S315080022B005D120210920C00600F0B8FD2AE0062C29
S315080022C005D140210920C00600F0B0FD22E0072C08
S315080022D005D180210920C00600F0A8FD1AE0082CC7
S315080022E004D101210D4800F0A1FD13E0092C04D109
S315080022F002210A4800F09AFD0CE00B2C04D11021AB
S31508002300064800F093FD05E00C2C03D18021034814
S3150800231000F08CFD204600F08FF810BD0004004840
S315080023207FB500200090019002900390002427E0DA
S3150800233000250CE0E800294940186100405AA10030
S315080023406A4651584018A1005050681C85B2142D91
S31508002350F0DBA1006A4650581421FFF7DBFA282162
S31508002360484361001E4A515A3C225143461864218B
S315080023703046FFF7CFFA6100194A5052601C84B202
S31508002380042CD5DB17488078002826D014484088C6
S315080023901549884203DC1248808888420ADD1148BC
S315080023A02038407A002805D11049486001210D4897
S315080023B0203841720A4840880A2803DB0848808882
S315080023C00A280ADA07482038407A002805D107493A
S315080023D0486001210348203841727FBD400400202F
S315080023E03C010020C0030020E60F0000C0010020C9
S315080023F000B587B001A800F0AFF80121480201F046
S3150800240009F80020019070200290012080020390B4
S3150800241000200690059001A9064800F031F8012130
S31508002420044800F021F80121024800F011F807B02D
S3150800243000BD00000024014010B504460723002211
S315080024402146024800F038F810BD0000002401407B
S31508002450002904D0426801231A43426003E0426817
S315080024605208520042607047002904D08268082347
S315080024701A43826003E0826808239A4382607047A1
S3150800248042680B4B1A4042600B684A681A43436815
S315080024901A4342608268074B1A4082600B694A6990
S315080024A01A438B681A4383681A4382607047000090
S315080024B00FBCFFFF8FF1F9FFF0B504460D4616462F
S315080024C01F463F073F0F2B46082B0FD91B071B0F2D
S315080024D0083B606F9A000F21914088436067606FE0
S315080024E099003A468A40104360670BE0206F9A00CD
S315080024F00F21914088432067206F99003A468A4009
S3150800250010432067E0680121A9408843E060E0683D
S315080025100121A9400843E0600120800328400028E3
S3150800252003D0012000F020F807E00120C00328406E
S31508002530002802D0012000F017F8F0BD002905D0C8
S315080025408268FF2301331A43826004E08268FF230E
S3150800255001339A43826070470021016041608160BF
S315080025600173016141617047002806D00649496830
S315080025700C221143044A516005E0034949680C22BC
S315080025809143014A516070470024014010B5244820
S315080025900078012834D10020214908702149088093
S315080025A012E02048008840001F49085A1F49098838
S315080025B0C9001F4A89181B4A1288520088521948AE
S315080025C00088401C17490880164800880428E8DB5C
S315080025D07E2001F00FFE022000F02EF90121154899
S315080025E0FFF7ACFF11480088401C104908800846D0
S315080025F00088142804DB0020088001200E49087092
S315080026000D480078002806D0FFF78AFE00200A4900
S31508002610087000F055FC7E2001F0ECFD10BD0000AE
S315080026204C010020660100200804002068010020F3
S31508002630400400200024014044010020FFB583B077
S315080026400C46029400200190002726E000261CE094
S31508002650721C039951430846791CFFF75BF9054636
S31508002660A54201D9281B00E0601B05460298A8422E
S3150800267004D90295059806700698077002980028EE
S3150800268002D10120019002E0761C402EE0D300BF63
S315080026900198002800D002E07F1C042FD6D300BF83
S315080026A0029807B0F0BD000000BF00BF00BF00BF22
S315080026B000BFBFF34F8F00BF00BF00BF06480749E2
S315080026C0C86000BF00BF00BFBFF34F8F00BF00BF89
S315080026D000BF00BF00BFFDE70400FA0500ED00E0FB
S315080026E010B500F001F810BD10B523480078002891
S315080026F017D1224800F016FF01283CD11F48007860
S31508002700002838DD1D480078402834DC01F05FFADF
S315080027101B490860012018490870002019490870EB
S3150800272029E0164A17490978491C501800F0FAFE9C
S31508002730012816D113480078401C124908700F4822
S3150800274000780978884216D100200B4908700B4892
S315080027504078FF280FD10B48007802280BD1FFF7E5
S31508002760A3FF01F034FA064909686431884202D9A0
S3150800277000200149087010BD15010020C40300207F
S31508002780180100201401002010B586B00446012166
S31508002790880300F03FFE0121480400F01BFE0122D9
S315080027A00921C80600F02DFB01220A210920C006CE
S315080027B000F027FB01A801F010FB019430216846C0
S315080027C0018100214181818101821821C18101A9EC
S315080027D0184801F0BFFA0121164801F098FA05A831
S315080027E000F065FB01214902684681820121817555
S315080027F01821C17505A90920C00600F0B5FA0121FE
S315080028008902684681824821C17505A90920C00642
S3150800281000F0AAFA1B2168460170032141700121C4
S31508002820817000F0A3FD01220221024801F087FA17
S3150800283006B010BD0038014001B50449009808608B
S3150800284000BF024800680028FBD108BD1C01002013
S31508002850014600220E4B1A61CA005A6100229A618B
S3150800286005221A6100BF0A4A1069C207D20F002A58
S3150800287004D0012212040240002AF4D0044A126944
S3150800288052085200024B1A6100229A6170470000F2
S3150800289000E000E010B500210448FFF74FFE0220D3
S315080028A000F04AF801200249087010BD00240140D2
S315080028B04C01002000B589B00121084600F08AFDC8
S315080028C01A4800F045F801A800F08EF8184801905B
S315080028D0184802900021684601730420049068464F
S315080028E00175802141754900C18289000183202133
S315080028F08176090281830021C183018401A90B48DD
S3150800290000F04CF80121094800F01CF801220221C8
S31508002910064800F039F8092168460170022141701D
S315080029200121817000F022FD09B000BD08000240B7
S31508002930002401400804002001494860704700004F
S31508002940000002400268520852000A4302607047BB
S3150800295010B504462068400840002060002020602A
S315080029606060A060E060E1B2084608380521FEF71D
S31508002970D1FF01460F2088400249496808430149AA
S31508002980486010BD00000240002A03D003680B43CC
S31508002990036002E003688B430360704710B50A7A48
S315080029A08B7D1A430B7C1A434B7C1A434B8A1A437A
S315080029B08B8A1A430B8B1A434B8B1A430368094CB1
S315080029C023401A43026002680123DB039A438B8B78
S315080029D01A430260CA6842600A6882604A68C2602E
S315080029E010BD00000F80FFFF0021016041600172E9
S315080029F0C16001744174418281828175018341837A
S31508002A008183704770B506460C4621460A4800F091
S31508002A104BF90546002D01D1401E70BD064885427A
S31508002A2002D10648051B00E02D1B224629463046E2
S31508002A30FEF79AFF2046F0E700F4000800FC0008BD
S31508002A4070B506460C4621460A4800F02DF905469B
S31508002A50002D01D1401E70BD0648854202D10648A8
S31508002A60051B00E02D1B224629463046FEF77CFF53
S31508002A702046F0E7008000080088000870B5064682
S31508002A800C4621460A4800F00FF90546002D01D1EB
S31508002A90401E70BD0648854202D10648051B00E067
S31508002AA02D1B224629463046FEF75EFF2046F0E7F4
S31508002AB0009000080098000870B505460C462246A6
S31508002AC00249284600F0B1F8204670BD00F4000817
S31508002AD070B505460C4622460249284600F0A5F878
S31508002AE0204670BD0080000810B5044608480069F5
S31508002AF002210843064908610846446100694021E5
S31508002B00084303490861034800F00EF910BD0000A8
S31508002B1000200240FF0F00000C48C068C007C00F25
S31508002B20002801D0012070470848C06804210840E1
S31508002B30002801D00220F6E70448C06810210840A2
S31508002B40002801D00320EEE70420ECE7002002402D
S31508002B50034800698021084301490861704700005D
S31508002B600020024030B504460D460548006901219B
S31508002B7008430349086125800F2000F0D5F830BDC9
S31508002B800020024010B57E2001F034FB064800F014
S31508002B900FF87E2001F02EFB044800F009F87E208D
S31508002BA001F028FB10BD000000F4000800800008B2
S31508002BB010B5044600F0ACF82046FFF795FFFFF77E
S31508002BC0C7FF10BD70B503460125002208E0500076
S31508002BD01C5A0748844201D0002506E0501C82B2E0
S31508002BE0CE0F761876109642F1DC00BF284670BDE7
S31508002BF0FFFF0000F8B505460E46144600F088F8B3
S31508002C007E2001F0F7FA002707E029883046FFF70B
S31508002C10A9FFB61CAD1C781C87B2E10F091949102B
S31508002C20B942F2DCFFF794FFF8BDF8B507460C4643
S31508002C3015462946204600F037F80646002E0DD1DF
S31508002C402046FFF7B5FF012080022018FFF7B0FFE6
S31508002C502A4621463846FFF7CDFF24E001208002A8
S31508002C602018401BB0420AD1012080022018FFF725
S31508002C709FFF2A4631463846FFF7BCFF13E001207E
S31508002C80C0022018401BB04208D12046FFF790FF2B
S31508002C902A4631463846FFF7ADFF04E02A46314654
S31508002CA03846FFF7A7FFF8BDF8B505460E462F4686
S31508002CB0E807C00F002801D000BFFEE73146012013
S31508002CC0C002FEF73DFE002901D000BFFEE7002442
S31508002CD00BE020467043471931463846FFF772FF26
S31508002CE0012800D108E0601C84B231460120C002E8
S31508002CF0FEF726FEA042ECDC00BF31460120C002EA
S31508002D00FEF71EFEA04200D100273846F8BD000097
S31508002D1002480349486003484860704723016745ED
S31508002D2000200240AB89EFCD10B5024600BFFFF781
S31508002D30F3FE0346521EFF2400E0641E002CFCD15D
S31508002D40012B01D1002AF2D1064800697721884370
S31508002D50044908613420C860002A01D1052010BD45
S31508002D601846FCE700200240F8B50246CD782F0742
S31508002D703F0FCD7810263540002D01D08D782F4392
S31508002D801446002011E085062B0E0D880126864084
S31508002D903540002D07D025680F269E40B5433E4690
S31508002DA09E4035432560451CE8B20828EBDB141D18
S31508002DB00D882D120095002011E085062B0E0125A1
S31508002DC08540009E3540002D07D025680F269E4079
S31508002DD0B5433E469E4035432560451CE8B2082863
S31508002DE0EBDBCD78282D04D155690E88354355611E
S31508002DF006E0CD78482D03D115690E88354315614F
S31508002E00F8BD70B54D07EB0E082902DA05462035E0
S31508002E1001E0054624352C460F269E402568B54315
S31508002E2016469E403543256070BD000038B50446F9
S31508002E300D460920C006844203D10121480400F04A
S31508002E40C9FA1148844203D10121000200F0C2FAEE
S31508002E500E48844203D10121000200F0BBFA0C4857
S31508002E60844203D10121080500F0B4FA684600F04F
S31508002E701EF868460580012181700021C1706946E7
S31508002E802046FFF771FF38BD0004004800080048D7
S31508002E90000C0048024690680840002801D001202E
S31508002EA070470020FCE741617047016170470021C7
S31508002EB0C9430180022181700421C1707047000056
S31508002EC0F0B58FB00025002600200D900C907E20CE
S31508002ED001F090F900241AE06100A34A505AFEF75F
S31508002EE0D8FFA2490790FEF7F9FD0746FFF72CF829
S31508002EF000229F4B09910890FEF7E0FE0B910A907D
S31508002F00FFF74AF8A1009B4A5050601C84B2042C73
S31508002F10E2DB98498868FFF717F8974A974B0591B7
S31508002F200490FEF7BDFE0022954B07910690FEF72A
S31508002F302DFF944A944B09910890FEF7B7FE0B9122
S31508002F400A90FFF729F805468A494868FEF7FCFF04
S31508002F50894A8A4B05910490FEF7A2FE0022884B07
S31508002F6007910690FEF712FF864A874B099108904B
S31508002F70FEF79CFE0B910A90FFF70EF806462846C8
S31508002F80FEF7E2FF00227A4B05910490FEF78EFECB
S31508002F900991089029467D48FEF763FD0746FEF726
S31508002FA0D3FF07910690099B089AFEF7EFFE0B914F
S31508002FB00A90FEF7F1FF764908603046FEF7C4FF2F
S31508002FC000226B4B05910490FEF770FE099108905C
S31508002FD031466E48FEF745FD0746FEF7B5FF0791F1
S31508002FE00690099B089AFEF7D1FE0B910A90FEF708
S31508002FF0D3FF684908606849088BFEF765FF674A8A
S31508003000674B03910290FEF759FE0022654B059126
S315080030100490FEF7BBFE099108905F49088BFEF7FE
S3150800302038FF0746FEF790FF00225E4B019100909D
S31508003030FEF7ACFE0591049055480068FEF784FF3C
S3150800304003910290059B049AFEF72AFE07910690C3
S31508003050099B089AFEF79AFE0B910A90FEF79CFFC9
S315080030600D904D49488BFEF72FFF4C4A4C4B039168
S315080030700290FEF723FE00224A4B05910490FEF7C4
S3150800308085FE099108904449488BFEF702FF0746DA
S31508003090FEF75AFF0022434B01910090FEF776FE99
S315080030A0059104903B480068FEF74EFF0391029095
S315080030B0059B049AFEF7F4FD07910690099B089A6A
S315080030C0FEF764FE0B910A90FEF766FF0C903648F1
S315080030D00D99FEF76DFC0746FEF704FF33490860B5
S315080030E031480C99FEF764FC0746FEF7FBFE3049AB
S315080030F008603048008A2D4909684018C003010C49
S315080031002C480182408A2A4909684018C003010CE4
S31508003110284841821749C8682749FEF7A2FC07468E
S31508003120FEF7E0FE81B223480184FF38C1380088E3
S31508003130FF21F531884215DD0020174950390880EE
S315080031400C4908681D49FEF743FF0BD21948203081
S31508003150407A002806D1104950394860012115489F
S31508003160203041720FB0F0BD3C01002000F07F45D1
S315080031700000084030040020333333333333C33F71
S315080031800000284025068195438BD43F000048431C
S31508003190540100205801002010020020091B9E5EE1
S315080031A029CB703F00408F400000C8415C010020D9
S315080031B060010020800300200000C8427B142E3FD7
S315080031C00148006870470000200100200348006895
S315080031D00349097840180149086070472001002012
S315080031E02801002008B50121480400F0F3F8012160
S315080031F0880400F0EFF86846FFF759FE0121C90375
S31508003200684601804821C17069460920C006FFF753
S31508003210ABFD6846FFF74BFE0121090368460180AE
S315080032204821C17069460920C006FFF79DFD68461A
S31508003230FFF73DFE4021684601800421C1706946BA
S315080032400148FFF791FD08BD0004004810B50121AB
S31508003250C9030920C006FFF71DFE002808D1234828
S31508003260807B002808D1012120488173C17103E0C1
S3150800327000211E48C17181731D4880681D49884216
S315080032802DD900201A49886000211848C1712030BC
S31508003290807800281DD108211748FFF706FE134835
S315080032A09038408803280CDA10482038408A82284B
S315080032B004DA01210D482030817002E001210B4813
S315080032C041720A488079012809D1002008494860D6
S315080032D005E00020064948600021044881717E20E7
S315080032E000F088FF0148C07910BD0000A003002047
S315080032F0C0010020DC0500000004004808B50121D3
S31508003300480400F067F80121880400F063F868466D
S31508003310FFF7CDFD29216846018001218170102122
S31508003320C17069461048FFF71FFD9621684601805F
S31508003330012181701021C17069460920C006FFF776
S3150800334013FD10210920C006FFF7ADFD80210920D5
S31508003350C006FFF7A8FD01210348FFF7A4FD0821D1
S315080033600148FFF7A2FD08BD00040048817800293E
S3150800337025D0174903221202891802789210920062
S31508003380895802789207D30EFF229A4091434278D1
S315080033909207120E03789B07DB0E9A4011430C4ADC
S315080033A003231B02D21803789B109B00D150017887
S315080033B0CA06D20E01219140054A116007E001783C
S315080033C0CA06D20E01219140014A80321160704727
S315080033D000E100E0002905D0054A52690243044B82
S315080033E05A6104E0024A52698243014B5A617047A6
S315080033F000100240002905D0054AD2690243044B51
S31508003400DA6104E0024AD2698243014BDA61704705
S3150800341000100240002905D0054A92690243044B70
S315080034209A6104E0024A92698243014B9A617047A5
S315080034300010024010B500F031F804494968F0223E
S3150800344011400909024A515CC84010BD00100240EB
S31508003450EE00002010B5FFF7EDFF05494968072281
S3150800346012021140090A034A515CC84010BD000007
S3150800347000100240EE00002010B5FFF7DBFF0549FB
S3150800348049680722D2021140C90A034A515CC8405A
S3150800349010BD000000100240EE000020F8B51E48DE
S315080034A040680C210840042802D008282ED101E0E3
S315080034B01A4C2DE0184840300069C007C00F002894
S315080034C00AD015484030006902210840002801D07A
S315080034D0134802E0114800E0104807460E484030FD
S315080034E00069FF2109040840000C451C0A484030C1
S315080034F00069072109020840000A461C3946694343
S3150800350008463146FEF706FA044601E0034C00BFBA
S3150800351000BF2046F8BD00000010024000127A00E5
S3150800352000093D0070B5044600250221074800F051
S31508003530F4FB002808D0054800F048FC207002215A
S31508003540024800F0E2FB0125284670BD003801401C
S3150800355010B500F001F810BD00B585B062480068E6
S31508003560012108436049086000BF5F4800680221DE
S3150800357008400028F9D05D485D4908605D48006844
S31508003580102108435B49086008460068C008C00067
S31508003590086057490968481E5749FEF7BBF9049061
S315080035A05448006804994907490F08435149086077
S315080035B04D484068514908404B49486008464068AC
S315080035C0902108434849486008464068486048488A
S315080035D000684649884207D94348406805210902D8
S315080035E00843414948600BE041480068444988421D
S315080035F006D93D4840680121890208433A4948608E
S315080036006B4601AA3A4801683E48FFF717F836485C
S315080036104030006980088000334940310861084617
S315080036200069400840000861684600784007400F76
S315080036300290684600794006400E03902A48C06901
S31508003640890508432849C8612748403000692E493A
S315080036500840254940310861039800040299090287
S31508003660084321494031096908431F494031086127
S315080036701D4800680121090608431B49086000E047
S3150800368000BF194800680121490608400028F7D0FC
S315080036901548406880088000134948600846406815
S315080036A0022108431049486000E000BF0E48406800
S315080036B00C2108400828F8D10120FFF7C9F80A4864
S315080036C0406810218843084948600120FFF7C0F880
S315080036D00548406880218843034948600120FFF770
S315080036E0B7F805B000BD00000010024000A24A0469
S315080036F0000100200020024000366E010FC0FFFFC7
S315080037000051250200127A00FFF800FF042806D1AE
S315080037100649096904221143044A116105E003496F
S31508003720096904229143014A1161704700E000E0EB
S3150800373010B5FFF74BFD4D480088401C4B490880E3
S3150800374008464068401C486049480068002804D07C
S3150800375047480068401E464908604648C07901281F
S3150800376005D142488068401C4049886002E0002034
S315080037703E4988603F480079012805D13B480069E1
S31508003780401C3A49086102E0002038490861394876
S31508003790807A012805D13548C06B401C3349C86377
S315080037A002E000203149C863304948680A21FEF71B
S315080037B0B1F800291CD12F48C17F807F814206DDE0
S315080037C02C48807F401CC1B22A48817710E02948DE
S315080037D0C17F807F814200D10AE02648C17F807F71
S315080037E0814205DA2348807F401EC1B2214881778D
S315080037F0204820308078022804D01E48203080785F
S31508003800032804D11948406B401C184948631948D5
S315080038102030007800280AD11648203080780428FD
S3150800382005D11248406C401C1049486402E000204B
S315080038300E4948640F48C07B012805D10B48C06C67
S31508003840401C0A49C86402E000200849C8640948BF
S31508003850007C012805D10548806C401C0349886412
S3150800386002E000200149886410BD0000C001002064
S315080038701C010020A003002010B51648006801218D
S315080038800843144908600846406813490840114926
S31508003890486008460068114908400E49086008460D
S315080038A000680121890488430A4908600846406877
S315080038B0C32109048843074948600846006808493F
S315080038C00840044908609F2000048860FFF740FE0E
S315080038D010BD0000001002400CC0FFF8FFFFF6FE06
S315080038E0FFFF8F0008B501214804FFF773FD022288
S315080038F001210920C006FFF784FA022168460180E3
S315080039001821C1700121817069460920C006FFF798
S315080039102BFA01214804FFF75DFD02221146092012
S31508003920C006FFF76EFA0421684601801821C170A7
S315080039300121817069460920C006FFF715FA08BDFE
S3150800394030B587B004460D4601210846FFF752FDFB
S3150800395004A800F033F9059468460582002101831E
S315080039608176817404A90120800700F0F1F8684681
S3150800397000F0D2F8602168460170012141700020EC
S31508003980019000216846017269460120800700F00F
S3150800399057F869460120800700F08AF80821C8060A
S315080039A000F07EF80821C80600F0B0F840210806A5
S315080039B000F038F84021080600F03CF80121880795
S315080039C000F00AF80121880700F01EF8012188078F
S315080039D000F00EF807B030BD002904D00268802335
S315080039E01A43026003E0026880239A430260704724
S315080039F0002904D0026801231A43026003E0026822
S31508003A005208520002607047002905D0426C012313
S31508003A10DB031A43426404E0426C0123DB039A4346
S31508003A2042647047826907231B039A430B021A43B1
S31508003A3082617047C26970239A430A43C26170471C
S31508003A4010B5826907231B039A430B781B021A4396
S31508003A5082610A7A12014B781B011A43036A3024E1
S31508003A60A3431A4302624A6882630C4A904213D1FE
S31508003A704A7A12018B781B011A43036AC024A343AE
S31508003A801A4302624A8992008B899B001A4343684B
S31508003A902401A3431A43426010BD0000002C0140D4
S31508003AA082690123DB029A430B021A43826170473B
S31508003AB010B5C26970239A430B781A43C2610A7A11
S31508003AC012024B781B021A43036A03242402A343F7
S31508003AD01A4302624A68C2630B4A904213D14A7A71
S31508003AE012028B781B021A43036AA400A3431A43E3
S31508003AF002624A8912018B891B011A434368A40092
S31508003B00A3431A43426010BD002C0140C269082332
S31508003B109A430A43C261704700210170417081705F
S31508003B204160017241724181818170470122920789
S31508003B30904201D1816301E08AB282637047012213
S31508003B409207904201D1C16301E08AB2C26370470D
S31508003B50026803231B029A430B891A430260134A1D
S31508003B60904206D001229207904202D0104A904213
S31508003B7005D1026870239A438B781A4302600B4A70
S31508003B80904205D00B4A904202D00B4A904205D18A
S31508003B90026B120A12028B7A1A4302634A68C262DD
S31508003BA00A8882620122426170470000002C0140A7
S31508003BB00004004000440140004801400021C94378
S31508003BC0416000210180018181708172704710B5C2
S31508003BD0FFF7F6FA10BD000070B5FFF72BFC054697
S31508003BE07D21C900FDF796FE0446601E0C498842F1
S31508003BF000D90CE0601E0B4948610321081F00F03C
S31508003C006FFB0020074988610720086100BF042070
S31508003C10FFF77CFD0021481E00F062FB70BD000026
S31508003C20FFFFFF0000E000E010B50221154800F094
S31508003C307DF8002824D0134800F0C8F8C4B212480A
S31508003C400079002803D1204600F052FF14E00E4800
S31508003C500079022810D10C48407900280CD10B486D
S31508003C608079AA2804D10948C471012106484171FE
S31508003C70AA2C01D1054884710221024800F045F8B2
S31508003C8010BD000000380140A0030020F004002009
S31508003C9010B504462146054800F09CF800BF0121EE
S31508003CA0024800F03AF80028F9D010BD0038014063
S31508003CB070B505460E4600247E2000F09BFA00BF2C
S31508003CC020E0042C19DD701EA04216DD285D7E2832
S31508003CD006D17D20FFF7DCFF5E20FFF7D9FF0FE056
S31508003CE0285D7D2805D1FFF7D3FF5D20FFF7D0FFBC
S31508003CF006E0285DFFF7CCFF02E0285DFFF7C8FF66
S31508003D00601C84B2B442DCDB70BD416170478269D5
S31508003D10520852000A43826170470246906808407A
S31508003D20002801D0012070470020FCE70246D06831
S31508003D300840002801D0012070470020FCE7002A2F
S31508003D4003D003690B43036102E003698B430361F4
S31508003D507047000070B504460D460026E06930211C
S31508003D60884329790843E061E06944218843A979B1
S31508003D700843E061E06980088000297A0843E06129
S31508003D80A0691821884369890843A061A0690421AC
S31508003D908843297B0843A0610B48844203D1FFF777
S31508003DA06BFB064602E0FFF755FB064630462968D8
S31508003DB0FDF7B0FD0009206230462968FDF7AAFD27
S31508003DC00007000F606270BD003801400146486870
S31508003DD0C0B27047CAB2026070474B21C901016080
S31508003DE03021017100218171017218214181002160
S31508003DF00173704710B51C484088030000F061FA4B
S31508003E000504111E292A2B0017487030008CFF2143
S31508003E101B31884204DA01211348418000F00AFA6E
S31508003E2019E011487030008CFF210531884204DA08
S31508003E3002210D48418000F0FDF90CE00A48703077
S31508003E40008CFD2804DA03210748418000F0F2F9C6
S31508003E5001E000E000BF00BF0348903080790028E9
S31508003E6001D100F0E7F910BD1003002010B5304865
S31508003E704088002806D0012813D0022820D003281D
S31508003E8054D12CE080210920C006FFF70EF8012145
S31508003E902848FFF70AF810210920C006FFF705F899
S31508003EA044E001212348FFF700F880210920C006D5
S31508003EB0FEF7F9FF10210920C006FEF7F4FF35E0EA
S31508003EC080210920C006FEF7F0FF01211948FEF7F8
S31508003ED0EAFF10210920C006FEF7E5FF26E016498D
S31508003EE04868CD21FDF716FDC007C00F002805D08C
S31508003EF080210920C006FEF7D6FF0DE00E49486866
S31508003F00CD21FDF707FDC007C00F002804D1802189
S31508003F100920C006FEF7C9FF01210648FEF7C3FFC0
S31508003F2010210920C006FEF7BEFF00BF00BF10BD66
S31508003F301003002000040048C001002010B5964870
S31508003F408078030000F0BDF90504336CAFFDFC0072
S31508003F5091482038008CFF210531884202DB012177
S31508003F608D48817040218D48FEF794FF00281DD0AA
S31508003F708B494868FF21F531FDF7CCFCC007C00F17
S31508003F80002805D180210920C006FEF78CFF04E031
S31508003F9080210920C006FEF788FF10210920C006E7
S31508003FA0FEF781FF01217D48FEF77DFFF2E07A48A2
S31508003FB02038008CFF211B31884202DB022176481B
S31508003FC0817040217548FEF765FF002827D074499F
S31508003FD04868FF21F531FDF79DFCC007C00F002892
S31508003FE004D101216D48FEF75EFF03E001216B480D
S31508003FF0FEF75BFF80210920C006FEF754FF10215B
S315080040000920C006FEF74FFF63489038408801280C
S3150800401005D0012160489038418000F00BF9B9E0DD
S315080040205D482038008CFF212531884202DD0321B6
S315080040305948817040215948FEF72CFF002831D095
S3150800404057494868FF21F531FDF764FCC007C00FE2
S3150800405000280ED180210920C006FEF726FF01217F
S315080040604E48FEF722FF10210920C006FEF71DFF65
S315080040700DE080210920C006FEF715FF1021092052
S31508004080C006FEF710FF01214448FEF70CFF424820
S3150800409090384088002805D000213F489038418054
S315080040A000F0C8F876E040213C48FEF7F3FE002809
S315080040B04ED0012109030920C006FEF7EBFE0028B1
S315080040C011D180210920C006FEF7EFFE01213348F1
S315080040D0FEF7EBFE10210920C006FEF7E6FE0421D6
S315080040E02D48817026E02E494868FF21F531FDF7F5
S315080040F011FCC007C00F00280ED180210920C00678
S31508004100FEF7D3FE01212548FEF7CFFE1021092030
S31508004110C006FEF7CAFE0DE080210920C006FEF79C
S31508004120C2FE10210920C006FEF7BDFE01211B486C
S31508004130FEF7B9FE184890384088002808D001E0F4
S3150800414027E006E0002114489038418000F072F814
S3150800415020E040211148FEF79DFE002818D0802156
S315080041600920C006FEF7A1FE01210C48FEF79DFEB8
S3150800417010210920C006FEF798FE074890384088A7
S31508004180002805D0002104489038418000F052F8F4
S3150800419000E000BF00BF10BDA003002000040048D7
S315080041A0C001002003488068400840000149886033
S315080041B070470000002C004080210143014A11602D
S315080041C070470000002C004003488068002801D092
S315080041D0012070470020FCE7002C004010B5FFF7CF
S315080041E0F3FF002804D0FFF7DDFF662000F002F891
S315080041F010BD00004106490E014A116070470000D3
S31508004200002C004004494968FF228132914301434A
S31508004210014A516070470000002C00400449496873
S31508004220C909C9014206520E1143014A5160704735
S31508004230002C004010B57E20FFF7DCFF0948FEF78A
S31508004240B7FC0949094801820521103000F09AF89F
S315080042500649103148814022024904481030FEF7C9
S31508004260E4FC10BD00900008FBAA00000003002033
S3150800427070B505460C460121C802FFF7BBF8FF20BA
S315080042808130FFF7BFFF2046FFF7C8FF2846FFF734
S3150800429093FF70BD2021020C01D010211046020A9E
S315080042A001D010460839020901D01046091F8208B4
S315080042B001D01046891E420801D0881E7047081A88
S315080042C0704730B47446641E2578641CAB4204D328
S315080042D0635D5B00E31830BC18471D46F8E700002D
S315080042E010B5002819DB1A4A03231B02D2188308C3
S315080042F09B00D2588307DC0EFF23A3409A438B0703
S315080043001B0E8407E40EA3401A43114B0324240210
S315080043101B198408A4001A5118E00E4A03071B0F3C
S31508004320083B9B089B00D2588307DC0EFF23A3405B
S315080043309A438B071B0E8407E40EA3401A43054BCA
S315080043400407240F083CA408A4001A5110BD000055
S3150800435000E100E01CED00E002E008C8121F08C1F9
S31508004360002AFAD170477047002001E001C1121FE8
S31508004370002AFBD170470000014908607047000019
S31508004380BC01002010B502460023002901D10020F7
S3150800439010BD03E01488921CE01883B208464C1E30
S315080043A0A1B20028F6D11846F2E70000F8B50027B2
S315080043B0002600240025F948407901286FD17E207F
S315080043C0FFF718FFF648C0790002F549097A08434D
S315080043D00746F348467A847A0246D17A107B00F07B
S315080043E0C5FC05460021ED484171EE49781A8F4211
S315080043F06FD01EDCEC49781A8F426BD010DCEB4983
S31508004400781A8F4267D006DC442F1CD0E848381843
S31508004410002872D1DEE1882870D08928F9D16FE1A9
S3150800442001286CD002286BD003286AD00428F0D162
S3150800443035E10300FFF745FF0C61C0FAF861611921
S3150800444026768E415C61062E09D1DA480078002866
S315080044500AD100F02FFF0120D649087004E0152E76
S3150800446002D1012000F026FFCFE1CC482030807829
S31508004470002806D0C9482038028A418A002000F060
S3150800448073FEC2E1002C0BD1C4482038408A0023B1
S315080044901A46F0210090FE2000F09BFE0CE0B5E1E4
S315080044A0012C09D1BD482038008A01230022F021B9
S315080044B00090FE2000F08DFEA7E1002C0CD1BE482E
S315080044C0408800231A46F3210090FE2000F081FE62
S315080044D00DE05AE056E188E1012C08D1B6488089FA
S315080044E001230022F3210090FE2000F072FE8CE1E9
S315080044F0002C07D1B048458006E085E114E11DE1AE
S315080045006AE07AE0AC488581AB488089FF21F531BD
S31508004510884206DA00F0CAFA0022FE21F42000F0EA
S315080045208CFE72E1002C09D1A348808800231A4624
S31508004530F1210090FE2000F04CFE0AE0012C08D183
S315080045409D48C08901230022F1210090FE2000F039
S3150800455040FE5AE1002C02D19748858003E0012CE1
S3150800456001D19548C58194488088FF21F531884254
S315080045700ADC9148C089884206DC00F097FA0022D6
S31508004580FE21F22000F059FE3FE1002C09D18A48AD
S31508004590C08800231A46E9210090FE2000F019FE83
S315080045A009E0012C07D1192001230022E9210090F6
S315080045B0FE2000F00EFE28E1002C01D17E48C580C1
S315080045C0FF202D30854206DA00F070FA0022FE211F
S315080045D0EA2000F032FE18E1002C0CD1764800895A
S315080045E06421484380B200231A46E2210090FE2047
S315080045F000F0EFFD00E000BF07E1002C06D16421C2
S315080046002846FDF79DF981B26B4801816A48008901
S31508004610FF21F531884206DC00F048FA0022FE2127
S31508004620E32000F00AFEF0E01EE0FFE7002C0CD1C4
S31508004630614840896421484380B200231A46EB2129
S315080046400090FE2000F0C5FD0DE0012C0BD15A4864
S31508004650008A6421484380B201230022EB2100909E
S31508004660FE2000F0B6FDD0E0002C07D164212846D4
S31508004670FDF766F981B25048418108E0012C06D160
S3150800468064212846FDF75CF981B24B48018200F0A7
S315080046900DFA0022FE21EC2000F0CFFDB5E0012C3A
S315080046A015D13E4890384088032807DA01213B484F
S315080046B02030817000204049503948600022FE2190
S315080046C0E42000F0BAFD01213448817117E0002C7E
S315080046D010D1002131488171203081700022FE21DD
S315080046E0E42000F0AAFD002032490870324950390A
S315080046F0486004E00022FE21E42000F09EFD84E0EC
S31508004700002C0FD12648C07A32280CDC2448C17AFE
S315080047102948418200F0CAF90022FE21DF2000F074
S315080047208CFD00E000BF70E02348408A00231A464B
S31508004730DE210090FE2000F04CFD66E0002C0FD133
S315080047401748C07A32281CDC1548C17A1A48818273
S3150800475000F0ACF90022FE21E12000F06EFD10E029
S31508004760012C0ED10E48C07A32280ADC0C48C17AD0
S315080047701148C18200F09AF90022FE21E12000F0DA
S315080047805CFD42E0002C19D10B48808A00231A46AA
S31508004790E0210090FE2000F01CFD1AE0A003002096
S315080047A0F0040020E9FE0000E0FE000056FE0000CE
S315080047B0AB01FFFFB801002010020020012C08D130
S315080047C01348C08A01230022E0210090FE2000F051
S315080047D000FD1AE0002C07D101210E4801710022C4
S315080047E002210D48FFF7ABFA0FE0002C0BD1FF2191
S315080047F001310A48FDF7D1F800200849891F0880C9
S3150800480002210448017100E000BF00BFF8BD0000A6
S3150800481010020020A003002000380140F604002002
S31508004820F0B589B00020089007900690384840797E
S3150800483001286BD137488079AA2864D13548C079D0
S31508004840322860DA3348C07900285CDD3149C979F5
S3150800485008461938FDF712FB08900898FDF774FB0F
S3150800486004462D4A2D4BFDF729FA00222C4B0191BF
S315080048700090FDF771F9039102902A480068FDF748
S3150800488063FB0646039B029AFDF780FA059104909E
S31508004890FDF782FB079024490798FDF7E2F80446DE
S315080048A0FDF720FB81B2214801830898FDF74CFBF0
S315080048B00646194A194BFDF701FA04460022184B19
S315080048C0FDF74AF90391029019480068FDF73CFB89
S315080048D001910090039B029AFDF758FA05910490FE
S315080048E0FDF75AFB069010490698FDF7BAF80446F4
S315080048F0FDF7F8FA81B20D48418300F0D7F8002198
S3150800490003480171817100210148417109B0F0BD68
S31508004910A0030020F0040020091B9E5E29CB703FEF
S315080049200000F03F5401002000007A4410020020E5
S315080049305801002070B505460E461446002E02D0D2
S31508004940012E4AD120E0002D02D0012D1AD10CE00B
S31508004950602101208007FFF765F800210120800704
S31508004960FFF7E4F81E4804700CE060210120800778
S31508004970FFF760F8002101208007FFF7E0F81948E3
S31508004980047000BF00BF28E0002D02D0012D22D1FF
S3150800499010E013480078A0420BD060210120800760
S315080049A0FFF740F8214601208007FFF7BFF80C48BB
S315080049B0047010E00B480078A0420BD0602101205B
S315080049C08007FFF737F8214601208007FFF7B7F879
S315080049D00448047000BF00BF00BF00BF70BD0000E0
S315080049E06A0100206B01002010B5052421E0802112
S315080049F02C48FCF7D2FF80212A48FEF703F80F213E
S31508004A002848FFF7BFFC2749C98B88420CD125489F
S31508004A101038008A2449884204D000F0CDF900F005
S31508004A2045F800E010BD04E0002000E0401C8028A6
S31508004A30FCDB2046611ECCB20028D8D100BF052475
S31508004A4023E080211748FCF7A8FF80211548FDF7C9
S31508004A50F7FF0F211348FFF795FC1249C98B8842C7
S31508004A600ED110481038008A0F49884204D000F049
S31508004A70A3F900F01BF802E000F018F8D2E704E00A
S31508004A80002000E0401C8028FCDB2046611ECCB2DA
S31508004A900028D6D100BF00F08FF900F007F800BF54
S31508004AA0C0E7000010020020FBAA000010B57E2017
S31508004AB0FFF7A0FBFEF766F80B490C4801820F21A9
S31508004AC01030FFF75FFC09491031C8838021074879
S31508004AD01030FDF7F1FF7E20FFF78CFB802103489D
S31508004AE01030FDF7F5FF10BDFBAA000000020020FC
S31508004AF070B5044600257E20FFF77CFB98480088A1
S31508004B00FA280ADD00209649088096490870FF2190
S31508004B1001319348801DFCF740FF92480078030056
S31508004B20FFF7CFFB08052031425BD5ECFDFC7E2C58
S31508004B3011D100208A49088001208A4908708848CE
S31508004B4001880088401C864A1080901D4454002025
S31508004B501146C87002E0002081490880002080497B
S31508004B600871FBE07E4801880088401C7C4A10805A
S31508004B70901D445402207B4908701046007900199C
S31508004B8011460871EAE0764801880088401C744A94
S31508004B901080901D4454032072490870104600790D
S31508004BA0001911460871D9E06D4801880088401C33
S31508004BB06B4A1080901D445404206A4908701046B8
S31508004BC000790019114608710846C470C078002893
S31508004BD002D1052063490870C0E061484079012880
S31508004BE056D15E2C1CD15E4800797E305C4908712E
S31508004BF07E215B4802880088401C594B1880981D06
S31508004C008154801FC078401EC0B21946C87000285B
S31508004C1002DC05205349087000205149487155E0C7
S31508004C205D2C1CD14E4800797D304D4908717D2197
S31508004C304B4802880088401C494B1880981D8154AF
S31508004C40801FC078401EC0B21946C870002802DC12
S31508004C5005204449087000204149487136E040481B
S31508004C60007900193E490871084601880088401CE9
S31508004C703B4A1080901D4454801FC078401EC0B225
S31508004C801146C870002821DC0520364908701DE049
S31508004C907D2C03D101203249487117E0304800794C
S31508004CA000192F490871084601880088401C2C4ABB
S31508004CB01080901D4454801FC078401EC0B2114613
S31508004CC0C870002802DC05202649087046E02448FA
S31508004CD00079C043401CC5B2A54203D1062021492C
S31508004CE0087002E007201F4908701D4801880088DF
S31508004CF0401C1B4A1080901D44542FE01848018818
S31508004D000088401C164A1080901D44547E2C0BD1F6
S31508004D100121154841710020114601E01DE00DE012
S31508004D2008801049087008E000200D490880002115
S31508004D300D48417100200B4908700FE00020094911
S31508004D400870074801880088401C054A1080901D95
S31508004D50445400201146088000E000BF00BF70BD23
S31508004D60F0040020B7010020A003002070B5024619
S31508004D70002013460C461D02FF2636023540254301
S31508004D80284670BD00BF00BF00BF00BF00BF00BF00
S31508004D9000BF00BF00BFFEE70549064801820021A3
S31508004DA0103041805F218180C180018170470000F9
S31508004DB0FBAA00000003002000B51349134801822E
S31508004DC0FF21103041800F210181A021C180D2210D
S31508004DD081801E214181AF21C1818C210182BE21A2
S31508004DE081810B4901830A49233141830521418287
S31508004DF00A218182C182002181830F21FFF7C2FA2D
S31508004E0002491031C88300BDFBAA00000002002039
S31508004E105A25000010B57E20FFF7ECF95648407A6F
S31508004E2001282AD15448807901281CD15349486859
S31508004E30C821FCF76FFDC007C00F002805D18021E7
S31508004E400920C006FEF72FF80DE04C494868C8212E
S31508004E50FCF760FDC007C00F002804D08021092098
S31508004E60C006FEF722F810210920C006FEF71BF837
S31508004E7001214348FEF717F810BD3F4880790128FD
S31508004E8078D13D4820308078002802D0012834D1D6
S31508004E900BE040213A48FDF7FDFF002802D1FEF756
S31508004EA0E5FF01E0FFF74AF863E034494868FF2167
S31508004EB0F531FCF72FFDC007C00F00280ED1802161
S31508004EC00920C006FDF7F1FF01212D48FDF7EDFF8A
S31508004ED010210920C006FDF7E8FF0DE08021092012
S31508004EE0C006FDF7E0FF10210920C006FDF7DBFF2D
S31508004EF001212348FDF7D7FF3BE01F482030807883
S31508004F00052827D11D494868FF21F531FCF702FD20
S31508004F10C007C00F00280ED180210920C006FDF762
S31508004F20C4FF01211648FDF7C0FF10210920C0065D
S31508004F30FDF7BBFF1CE080210920C006FDF7B3FF83
S31508004F4010210920C006FDF7AEFF01210C48FDF728
S31508004F50AAFF0DE080210920C006FDF7A6FF012162
S31508004F600748FDF7A2FF10210920C006FDF79DFF9F
S31508004F7000BF00BF00BF7FE7A0030020C0010020DC
S31508004F8000040048FEF778FCFEF7B8F9FDF792FC36
S31508004F90FDF72EFA0B20FDF75DF90C20FDF75AF9FF
S31508004FA00920FDF757F90320FDF754F90121564862
S31508004FB0FDF7C4FA4B200002FDF7E6FBFEF712F9EF
S31508004FC0FEF790FC0D216320FEF7BAFC01214F483D
S31508004FD0817100214172FFF707FDFEF7FDFD00F024
S31508004FE09DF8FEF743FF7F217E20FFF741F98AE00F
S31508004FF04648007900280AD1FDF7C8FAFFF70AFFE4
S31508005000FFF7D4F9FEF722F900F066FF78E03F488B
S315080050100079012836D1002301221946184600F0E6
S31508005020A9F900231A461946184600F0A3F9384884
S3150800503040683849884204D908213748FDF733FFC4
S315080050401DE033494868FF21F531FCF763FCC007CA
S31508005050C00F00280ED180210920C006FDF723FFC6
S3150800506010210920C006FDF71EFF01212A48FDF779
S315080050701AFF04E010210920C006FDF716FFFDF708
S315080050802FFB3DE021480079022839D1FDF77EFA49
S31508005090FEF7DCF8002301221946184600F06AF9E3
S315080050A000231A461946184600F064F9184840685D
S315080050B01849884204D908211748FDF7F4FE1DE06F
S315080050C013494868FF21F531FCF724FCC007C00FD7
S315080050D000280ED180210920C006FDF7E4FE102124
S315080050E00920C006FDF7DFFE01210B48FDF7DBFEB0
S315080050F004E010210920C006FDF7D7FEFFF790FB54
S315080051007E20FFF777F873E700240140A00300200C
S31508005110C0010020204E00000004004810B54021C0
S315080051200F48FCF73AFC40210D48FDF7A7FC05217E
S315080051300B48FFF727F90A49498988420AD10848DE
S315080051401038008A0749884208D0FFF725FEFFF77E
S3150800515071F803E0FFF720FEFFF76CF810BD0000BA
S3150800516010030020FBAA0000F7B5A0B00C461546B0
S3150800517080216846FCF711FC002700267E21684638
S315080051800170FE214170EF2181700721C1702099BD
S3150800519001710021417184712112C17101210172CD
S315080051A0457229128172012605E06846805DC0199C
S315080051B0C7B2701CC6B20B2EF7DBF843401CC1B24F
S315080051C06846C1727E2101730D21FEF771FD23B079
S315080051D0F0BDFFB585B005460E460E9F002001902E
S315080051E0029003900490009000247E216846017185
S315080051F0457186710421C171079901720899417236
S3150800520087723912C172012407E001A8015D00986E
S315080052100818C0B20090601CC4B2082CF5DB0098D0
S31508005220C043401CC1B2684601737E2141730A21FE
S3150800523001A8FEF73DFD09B0F0BDF7B584B00546F7
S315080052400E4600200090019002900390002700244B
S315080052507E2168460170467085700121C1706946D5
S3150800526006980871012405E06846005DC019C7B2B2
S31508005270601CC4B2052CF7DBF843401CC1B2684673
S3150800528041717E2181710721FEF712FD07B0F0BD3D
S3150800529070B504460D467E20FEF7ACFF03E0207885
S315080052A0641CFEF7F5FC2846691E8DB20028F6D167
S315080052B070BD000030B5A1B00446802101A8FCF7F6
S315080052C06CFB0025002C02D0012C20D10FE07E219A
S315080052D06846017100214171442181711321C17110
S315080052E01522104902A8FCF73FFB192510E07E217C
S315080052F068460171FE214171442181713321C171D2
S315080053003622094902A8FCF72FFB3A2500E000BF20
S3150800531000BF802D03DA294601A8FFF7B9FF21B09F
S3150800532030BD00006C01002081010020F8B506465A
S315080053300C46FCF72BFF051E0F4600D00120014343
S3150800534049000B484908411AC90F0DD0002E01D053
S31508005350012100E000210C4361004908401AC00FF2
S3150800536002D10120FFF708F828463946F8BD0000A3
S315080053700000F07FFFB58DB005460E4617460020A3
S315080053800B9000240A9009900890F9480078642840
S3150800539003D0F848C07F642803D10121F5488172FB
S315080053A002E00021F3488172002F02D0012F78D144
S315080053B028E2F148C089B04202D1EF48C48A00E029
S315080053C00524052C01DC052402E0322C00DB05242B
S315080053D0301BA8420DDDE748C07B00284CD1E648C3
S315080053E050384068E449503988610121E148C17361
S315080053F042E03019A8423FDCDE48C07B01283BD199
S31508005400DC482030007801282FD1DB485038406826
S31508005410D94950398969401AD84988420DD2D548A0
S3150800542090380089462820DDD24890380089801EA9
S3150800543081B2D0489038018117E0CF48503840688B
S31508005440CD4950398969401A7D21890188420CD98C
S31508005450C848903800895F2807DAC6489038008916
S31508005460801C81B2C348903801810121C14820308F
S31508005470017000212038C173BE48C07B012875D150
S31508005480301BA84273DDBC48503840687D21C900EE
S31508005490884207D26420B64908700021B54841748D
S315080054A0A9E1FDE3B348407C002869D10121B14850
S315080054B04174B148808964285ADAAE482038018A8E
S315080054C0408B081A81B2AB48203881830146888B05
S315080054D0FCF7DFFC01460690A9480068FCF7FEFACF
S315080054E00790FCF731FDA74A03C2A2492039098C67
S315080054F049430846FCF7D4FC07910690A1480CC816
S315080055000698FCF7DBFB9F4A03C29E4903C9FFF7CF
S315080055100DFF07910690FCF73FFD9B4908609549EA
S315080055202039088CFCF7B5FC0146059096480068BA
S31508005530FCF7D4FA95490690FCF793FA0790FCF71E
S31508005540D1FC934908700846007864280ADC8C4820
S315080055500068FCF7F9FC00228E4B07910690FCF7D1
S3150800556007FD08D864208A49087004E040E15BE03A
S315080055706420874908707F482038018A01873AE104
S315080055807D485038406C7D21C900884247D90020A3
S315080055907949503948647E48007864283BDA75486A
S315080055A02038018A008F814230DD0121890774483D
S315080055B00068FCF7FDF90790FCF794FC81B26D488A
S315080055C02038028A008F101A814205DA704800785E
S315080055D0801E6F4908701EE0664920390A8A098FBD
S315080055E0501AFCF74BFC0790654801680798FCF7CA
S315080055F0EFFC10D266480078801C6549087008469A
S315080056000078642807DD6420087004E060480078A4
S31508005610401D5F49087057482038018A01875C4851
S31508005620007853490870E6E0524820300078002890
S3150800563075D151488089642803DB64204C49087079
S31508005640D9E04D48503840687D21C900884206D2C5
S31508005650642047490870002146484174CBE0454814
S31508005660407C00285CD10121424841744248808927
S3150800567064284CDA3F482038018A408B081A81B2E0
S315080056803C48203881830146888BFCF702FC01469A
S3150800569006903B480068FCF721FA0790FCF754FC93
S315080056A0384A03C233492039098C49430846FCF76E
S315080056B0F7FB0791069033480CC80698FCF7FEFAE4
S315080056C0304A03C22F4903C9FFF730FE07910690F7
S315080056D0FCF762FC2C49086026492039088CFCF73F
S315080056E0D8FB0146059028480068FCF7F7F92749D2
S315080056F00690FCF7B6F90790FCF7F4FB2449087006
S3150800570008460078642805DD6420087002E06420F5
S315080057101F49087017482038018A01876BE061E045
S3150800572015485038406C7D21C900884255D900205B
S315080057301149503948640F482038018A008F814240
S3150800574043DD012189070E480068FCF731F9079007
S31508005750FCF7C8FB81B207482038028A008F101A66
S31508005760814219DA0A480078801E0949087031E032
S31508005770EA000020A0030020100200207017000095
S31508005780CC000020D0000020D80000200000C8422D
S31508005790E90000200000F03FFE490A8A098F501AE6
S315080057A0FCF76CFB0790FC4801680798FCF710FCAF
S315080057B010D2FA480078801CF84908700846007824
S315080057C0642807DD6420087004E0F4480078401D6A
S315080057D0F2490870EF48018A0187F0480078F049D5
S315080057E0087008E0EB487038007AED49087002E066
S315080057F00020EB490870EA48027838461099FFF706
S3150800580099F859E3E3484030807801285BD1E548A8
S315080058104088B04202D1E348448A00E00A24E148BD
S315080058204188408A081AA84209DBDE485038406891
S31508005830DC49503988620020DB4908701AE0D948EB
S315080058404088A84216DCD8480078002812D1D148EA
S31508005850018C41870120D4490870D24850384068E5
S31508005860D0495039896A401ACE49503908620846E3
S3150800587040680863CB488188808A081AA84209DBF1
S315080058800020CA490870C74850384068C549503989
S31508005890C8623CE0C3488088A84238DCC348007820
S315080058A0002834D1BB48018C81870120BF49087084
S315080058B0BC4850384068BB495039C96A401AB9498A
S315080058C05039486223E0B34840308078022808D12E
S315080058D0B4484088B04202D1B248448A17E00A2444
S315080058E015E0AC4840308078032808D1AD48808858
S315080058F0B04202D1AB48848A09E00A2407E0A948E5
S315080059008088B04202D1A748848A00E00A24052C80
S3150800591001DC052402E0322C00DB3224301BA842CD
S3150800592019DBA048503840689E495039C8610020A4
S31508005930486388639748C5832030007C002805D1D2
S315080059401E21944820308177012101740021914855
S31508005950203041733FE13019A842FBDC8D482030E6
S31508005960007C0128F6D18B484030807801287CD10C
S315080059708848403040780028F9D18A48408A0A2861
S315080059800BDB88495039086AFCF783FA884907907F
S31508005990FCF7A4F8874908601EE08248408A0A286E
S315080059A00FDA8048408A07280BDD7E495039086A95
S315080059B0FCF76FFA80490790FCF790F87D49086074
S315080059C00AE078495039086AFCF763FA7B49079078
S315080059D0FCF784F8774908606E49488FFCF759FA4E
S315080059E06C490690488FFCF754FA04907148016890
S315080059F00498FCF736F805900699FCF732F80790F4
S31508005A00FCF7A2FA6E4A03C26249488FFCF75CFAB1
S31508005A10039102906A4903C9FFF788FC0191009037
S31508005A20039B029AFCF7B2F90022664B0591049093
S31508005A30FCF744F907910690FCF768FA81B25548D5
S31508005A407038818057495039486AFCF722FA5A4912
S31508005A500790FCF743F8574908604E49888FFCF7CA
S31508005A6018FA4C490690888F00E05AE0FCF711FABC
S31508005A700490504801680498FBF7F3FF05900699CF
S31508005A80FBF7EFFF0790FCF75FFA4D4A03C241495F
S31508005A90888FFCF719FA03910290494903C9FFF761
S31508005AA045FC01910090039B029AFCF76FF90022CE
S31508005AB0444B05910490FCF701F907910690FCF711
S31508005AC025FA81B233487038C180364880896428FF
S31508005AD023DA34498889FCF7DCF9324950390690CB
S31508005AE0086BFCF7D6F938490290FBF7F7FF2D4902
S31508005AF004904A882749098B501AFCF7BFF9039086
S31508005B000499FBF7EBFF05900699FBF7AAFF2F49C7
S31508005B100790FBF7E3FF2049086001211D48403044
S31508005B2041702048503840681E495039C969401AA2
S31508005B302749884224DD17484030807802280DD14D
S31508005B401448703880885F281ADA124870388088B6
S31508005B50801C81B20F487038818011E00D484030B2
S31508005B60807803280CD10B487038C0885F2807DA7C
S31508005B7008487038C088801C81B206487038C180D1
S31508005B800021044820300174FF38E138406805498F
S31508005B9050391FE080030020CC000020E9000020D7
S31508005BA0EA00002010020020DC000020DD000020B2
S31508005BB000803B45C40000200000FA440080BB4436
S31508005BC0E00000200000594000007A440000C84266
S31508005BD070170000C861BA48007C01287ED1B84811
S31508005BE0807FB8490978884203DA0021B44881776A
S31508005BF04FE1301BA84205DD6421B148C177012178
S31508005C00817246E1AE4820308078012804D0022807
S31508005C1013D003287ED199E03019401BA04208DA38
S31508005C203019401B201A5F21081AC1B2A448C1774F
S31508005C3002E05F21A248C177FEE0A348406BA24973
S31508005C40896B401A7D21C90088424BD99E48406B12
S31508005C509D4988639A482038C08BA8420FDD98482A
S31508005C60903880880A3081B2954890388180C088FB
S31508005C70642832DB642192489038C1802DE090492F
S31508005C802039C98B691AE20F12195210521C914217
S31508005C9011DA8B4890388088801C81B2884800E0E9
S31508005CA00AE190388180C088642816DB642184481C
S31508005CB09038C18011E082492039C98B691AE20FF0
S31508005CC012195210921C914207DD7D48903880883F
S31508005CD0801E81B27A489038818000E0ADE078482D
S31508005CE02038C5837848406B784988420BD900200C
S31508005CF0754948638863724890388088401D81B228
S31508005D006F48903881806E48903801799030C17715
S31508005D106D4800E08CE040686B49C969401A6B49D8
S31508005D20884212DD664890388088401D81B26448F2
S31508005D3090388180C088642803DB642160489038E5
S31508005D40C180614840686049C86175E05E48406B3B
S31508005D505D49896B401A7D21C900884247D95A484E
S31508005D60406B5949886356482038C08BA8420FDDD6
S31508005D7053489038C0880A3081B251489038C1805B
S31508005D80C088642830DB64214D489038C1802BE0F8
S31508005D904B492039C98B691AE20F12195210521C45
S31508005DA091420FDA46489038C088801C81B2444830
S31508005DB09038C180C088642816DB64214048903832
S31508005DC0C18011E03E492039C98B691AE20F1219C0
S31508005DD05210921C914207DD39489038C088801EBF
S31508005DE081B237489038C18035482038C583344851
S31508005DF0903881799030C177334840683249C9690B
S31508005E00401A3349884212DD2D489038C088401D13
S31508005E1081B22B489038C180C088642803DB64218E
S31508005E2027489038C180284840682749C86103E058
S31508005E3032212348C17700BF2BE0214820308078E3
S31508005E40012823D13019A8421CDB1D489038017956
S31508005E509030C1773019801EA8420FDD1D480078A2
S31508005E60002816D1164890388088401D81B21448FB
S31508005E70903881800120174908700AE000201549EA
S31508005E80087006E000210E48C17702E00A210C4896
S31508005E90C1770B4820308078012806D10848C27F90
S31508005EA038461099FEF746FD05E00548827F3846D4
S31508005EB01099FEF73FFD00BF00BF0B9811B0F0BD6B
S31508005EC0A0030020EA000020C0010020881300007B
S31508005ED0581B0000E800002010B5F7488078002815
S31508005EE072D0F5484038408AFF217D31884204DC6B
S31508005EF0F1484038008A88420ADDEF482038407A5F
S31508005F00002805D1ED4948600121EB482038417247
S31508005F10EA48C06BEA4988420AD9E7482038407AF5
S31508005F20002805D1E54948600121E3482038417237
S31508005F30E1482038C07B01281ED1E048C06CE14901
S31508005F4088421DD90020DD49C864DB484038C18A2B
S31508005F50008A81420BDBD8482038407A00280FD1C6
S31508005F60D64948600121D4482038417208E0D24811
S31508005F704038018AC18203E0CF484038018AC1828D
S31508005F80CD482038007C01281FD1CC48806CCD49EB
S31508005F9088421ED90020C9498864C7484038818A82
S31508005FA0408A81420BDBC4482038407A002810D149
S31508005FB0C24948600121C0482038417209E0BE48FC
S31508005FC04038418A818204E036E0BB484038418A3D
S31508005FD08182B9482038407A01282DD1B648203820
S31508005FE08079012828D10023012219461846FFF78F
S31508005FF0C1F900231A4619461846FFF7BBF9AF48F8
S3150800600040687D210901884215D90020AB494860BE
S3150800601010210920C006FCF746FF80210920C0068A
S31508006020FCF741FF0121A848FCF73DFF0021A248E3
S3150800603020388171417210BD9F4820388079002828
S315080060405ED110210920C006FCF72DFF802109200A
S31508006050C006FCF728FF01219B48FCF724FF002116
S31508006060954881700023012219461846FFF782F9E0
S3150800607000231A4619461846FFF77CF98F484068E8
S31508006080FF21F531884204D220218F48FCF70DFF05
S3150800609025E220218C48FCF706FF88484068894994
S315080060A08842F5D984482038807B002817D1834850
S315080060B040687D214901884201D2FDF79BFE0821EF
S315080060C08148FCF7F0FE00217B48203841722030D9
S315080060D00170417000207949086208630BE040218D
S315080060E07948FCF7D7FE002805D000217248817050
S315080060F00121203881717D20400170494860EEE118
S315080061006D4880780300FEF7DCF8060457AEF3F115
S31508006110F0560021684801704170002067490862FE
S3150800612008630023012219461846FFF723F90023BE
S315080061301A4619461846FFF71DF95F484038418A3E
S31508006140018320300079012809D15C4800695F493C
S31508006150884203D900215848203801716BE757480F
S3150800616040687D210901884221D9002053494860A9
S3150800617040215548FCF78EFE002809D1FDF73AFE66
S3150800618008215148FCF78FFEFF20F530FCF754FB39
S3150800619010210920C006FCF786FE80210920C006CA
S315080061A0FCF781FE01214848FCF77DFE03E0082143
S315080061B04548FCF77AFE91E140484068FF21F531F1
S315080061C0884204D220214048FCF76FFE03E02021D4
S315080061D03D48FCF768FE394948687D21C900FBF748
S315080061E099FB23281FD2354948687D21C900FBF74A
S315080061F091FB192817D930484038018AFF38713879
S315080062004088814207DA2C484038418AFF3871387D
S315080062104088814216DB002028494860C86102216F
S31508006220254881700EE0254948687D21C900FBF79D
S3150800623071FB232806D3002020494860C861022143
S315080062401D4881701D4A50325188FF327132508A7A
S3150800625001231A46FFF78EF800231A4619461846F0
S31508006260FFF788F83AE115484068FF21F53188427A
S3150800627004D220211448FCF718FE03E02021124816
S31508006280FCF711FE0D484168503000897D22D20086
S31508006290504381421CD2094A50325188FF3271322A
S315080062A0508A01231A46FFF765F800231A4619464D
S315080062B01846FFF75FF817E0C0030020C00100206A
S315080062C070110100B80B0000000400488813000094
S315080062D000218548017400208449486001218248CC
S315080062E04173032120308170F8E086E043E0FFE740
S315080062F07D482038408AFF217D31884204DC7A486F
S315080063002038008A88420CDD0023012219461846E7
S31508006310FFF730F800231A4619461846FFF72AF8F9
S3150800632028E0724948687D21C900FBF7F3FA6F49EE
S3150800633050314989884210D26C4A50329188FF32CE
S315080063407132508A01231A46FFF714F800231A46B9
S3150800635019461846FFF70EF80CE063482038018AFC
S31508006360418300206149486000215F480174042187
S3150800637020308170B2E05C482038408AFF217D31A8
S31508006380884204DC58482038008A88420CDD0023FD
S31508006390012219461846FEF7EDFF00231A4619464C
S315080063A01846FEF7E7FF27E0504948687D21C900EF
S315080063B0FBF7B0FA4D495031098A0F39884214D291
S315080063C04A4A5032D189FF327132108A012300229B
S315080063D0FEF7D0FF454A5032D188FF327132508AD3
S315080063E001231A46FEF7C6FF06E000203F4948602B
S315080063F005213D482030817070E03C484068FF2107
S31508006400F531884204D220213948FCF74EFD0FE0C9
S3150800641036484068FF21F531884209D93348406833
S315080064204B21C900884203D220213148FCF73BFDA5
S315080064302E4840682F4988422DD22B482038408A5A
S31508006440FF217D31884204DC27482038008A8842AB
S315080064500CDD0023012219461846FEF78BFF0023A0
S315080064601A4619461846FEF785FF36E01F4A503287
S31508006470D189FF327132108A01230022FEF77AFF92
S315080064801A4A5032D188FF327132508A01231A468D
S31508006490FEF770FF21E020211548FCF706FD13489A
S315080064A040681549884218D30020104948600021E1
S315080064B00D48203081702038817100230122194649
S315080064C01846FEF757FF00231A4619461846FEF7E0
S315080064D051FF20210648FCF7E6FC00BF00BF7E20DE
S315080064E0FDF788FE00BFA6E5A0030020C001002036
S315080064F000040048A4380000983A00001C6500080B
S31508006500C000002000010000584300081C6600086F
S31508006510C001002038080000684300080000000099
S31508006520000000000000000000000000000000005D
S31508006530000000000000000000000000000000004D
S31508006540000000000000000000000000000001023A
S3150800655003040102030406070809000000A24A040E
S3150800656000000000000000000102030406070809F5
S31508006570000000000000000000000000000000000D
S3150800658004000000010000000000000000000000F8
S3150800659000000000000000000000000000000000ED
S315080065A000000000000000000000000000000000DD
S315080065B000000000000000000000000000000000CD
S315080065C0000000000000000000011058594C4C3033
S315080065D03131327878787878787878CB7E000110FF
S315080065E058594C4C303131327878787878787878D0
S315080065F004013205054C4C3031310614594132300C
S3150800660030353238483435303432417878787878CD
S311080066107D5D7E00000000000000000018
S705080018C515
